:020000040000FA
:1000000083161F30850000308800831280308800FE
:1000100031204030880031202030880031201030DD
:1000200088003120083088003120043088003120D9
:1000300002308800312001308800312002308800F1
:100040003120043088003120083088003120103001
:100050008800312020308800312040308800312055
:10006000062864308C00FF308D0014308E000000B4
:100070000000000000000000000000000000000080
:1000800000008E0B37288D0B35288C0B3328080089
:02400E00F93F78
:00000001FF
